:020000040000FA
:020000000528D1
:06000A00031383128501BF
:1000100086018316BF308500E230860006309B00E3
:1000200000309F00831289309F008316C0309400F7
:1000300083122030940013082310851D2328831673
:1000400085118312231406148615861596218611B0
:100050000130782101307821861585110130782111
:10006000013078218515051E3628CB2886110230EF
:10007000782100307821003078215530782186159C
:100080007F218611033078210030782100307821DB
:10009000FF3078218615553C031D532805179621FE
:1000A0009621051356289C219C219C21962196215E
:1000B000231C7A2885110230782100307821003005
:1000C00078215530782185157F21851103307821DD
:1000D0000030782100307821FF3078218515553C9B
:1000E000031D772805179621962105137A289C2150
:1000F0009C219C210610353078215030782106143F
:1001000096219621962106103A307821A030782148
:10011000061496219621962106103F307821F03062
:1001200078210614962196219621AF01FA30B1006C
:10013000003090000C10FF308F0012308E00101431
:10014000A321AD00AE010310AD0DAE0D0310AD0D3A
:10015000AE0D0310AD0DAE0D0310AD0DAE0D2E089E
:100160003038AE0006102E0878212D0878210614AC
:10017000AF0A2F08143C031DC128AF01B10BC128E1
:10018000C4280C1CC1289828902190219528A601EC
:10019000A701A901AA011F08C73910389F00003024
:1001A00090000C10851ED928FE308F004E308E0036
:1001B000DE28FD308F00A3308E00000010142708C9
:1001C000AC002608AB002A08AC02031CAB032908CC
:1001D000AB02231CEC28EE288611F128AB1FEC287B
:1001E0008511033078212B0878212C087821FF30E5
:1001F000782186158515AD00A70AA7080319A60A58
:100200001F15AE010310AD0DAE0D0310AD0DAE0DFB
:100210000310AD0DAE0D0310AD0DAE0D2E08303830
:10022000AE0006102E0878212D08782106141F191B
:1002300017291E08A8001F08C73908389F00231C6B
:100240002229242986112729A61F22298511023057
:100250007821260878212708782128087821861512
:1002600085151F151F1932291E08A900AA01231878
:100270003C290310A90CAA0C0608A4000310A40C26
:10028000A40E0F30A405073024020319602906309C
:100290002402031963290530240203196629043056
:1002A0002402031969290330240203196C2902303E
:1002B000240203196F2901302402031972297529B8
:1002C0000310A90CAA0C0310A90CAA0C0310A90C6A
:1002D000AA0C0310A90CAA0C0310A90CAA0C031059
:1002E000A90CAA0C0310A90CAA0C0C1C7529CB286C
:1002F00093008316141C7A29831213080800F9301E
:10030000A00000000000000000000000000000004D
:10031000A00B812900000000000000000000080080
:10032000FA30A1007F21A10B922908000830A20019
:100330009021A20B98290800051790219021051300
:100340009021902108002F08B000AF30B007013095
:100350000318013E8A003008AE21080082007F3475
:10036000A634CA34E634F834FE34F834E634CA34F9
:10037000A6347F3458343434183406340034063408
:0603800018343434583437
:02400E00033F6E
:02401000FC3F73
:00000001FF
